:1000000025006400A305070B8703F00E28000602F5
:100010000F0E2801100C240010022200000809070E
:10002000180C08063000050C3200A305140222004B
:10003000210CF202180C08070F0C3000A305140263
:10004000220008072A0C300073000A0C3200A305B6
:10005000140222003103F104330C0806420C300074
:10006000A30514022200350C2D0AF105B3023E0C43
:100070000806420C3000A30514022200400C2D0A91
:100080000F0C2D0AF20000004B0C08072A0C300060
:10009000A305140222004D0C450AF2021304560C6B
:1000A00008070F0C3000A30514022200580C500A58
:1000B000610C1307210C08070F0C3000A305140274
:1000C000220000000905510A000828000000E8028B
:1000D000660A00080409070C65090409070C65098C
:1000E0000409070C65090409020C650900000008F1
:1000F00004090F06EF0AAA026A040A02E201870A4B
:10010000940AA10AAE0ABB0AC80AD50AE20A09077C
:10011000F10A0904640011022B00A405C405900132
:10012000D80243070F05F40A2907F10A29046400DD
:1001300015022B00A405C4059101D90243070F0540
:10014000F40A4907F10A4904640019022B00A405C6
:10015000C4059201DA0243070F05F40A6907F10AA0
:10016000690464001D022B00A405C4059301DB0291
:1001700043070F05F40A8907F10A89046400A405FE
:1001800011022B00C4059401DC0243070F05F40A99
:10019000A907F10AA9046400A40515022B00C405EF
:1001A0009501DD0243070F05F40AC907F10AC904E6
:1001B0006400A40519022B00C4059601DE02430762
:1001C0000F05F40AE907F10AE9046400A4051D0219
:1001D0002B00C4059701DF0243070F05F40A010C49
:1001E0006509010C6509F40AA706EC02FA0A000089
:1001F0006409FC0A6409780A0409060C6509000010
:1002000087056A094F048F042F060E0B0F06110B8A
:100210004F05A7068F0500000000140B0F078F0580
:10022000130BA7074F0564090F0227006A094F0641
:100230006D0B800C2D00090C2E0064098F050D0636
:100240008F040F0227006A0903052D030000EE0248
:100250001D0B010C650987056A09FF0C0F060A02D0
:100260002D000A0C2E0064098F050D068F040F0265
:1002700027006A0903052D030000EE02330B010C71
:10028000650987056A090A0C2E000B020F07600B2F
:100290002D0064098F050D068F040F0227006A09DF
:1002A00003052D030000EE02490B0F04700CCA0178
:1002B00024000B022000080CE401C90C2000830B71
:1002C0006409640987046A09000000000000EE0266
:1002D000600B0000010C6509830B1F0C2E006F05DD
:1002E0008F05A7078F040F026F064F028F066F045A
:1002F00027006A09000000000000EE02700B87046E
:10030000010C6509830B0409A405C405D802F80093
:10031000D902F900DA02FA00DB02FB00DC02FC0081
:10032000DD02FD0064001102A405C4059001D8029D
:1003300043079B0B090464001502A405C405910141
:10034000D9024307A40B2904000004096400190220
:10035000A405C4059201DA024307AF0B4904640007
:100360001D02A405C4059301DB024307B80B690411
:10037000C4041102C40594012F04A7062F05DC0252
:100380004307C30B8904010C2F06380C2C00040909
:100390006400A4051502C4059501DD024307D10BD5
:1003A000A904DE02FE00DF02FF00C4041902C40536
:1003B0009601DE024307DD0BC904C4041D02C40517
:1003C0009701DF024307E50BE90400000000780A0B
:100400002907080C28063400050C360018022200C3
:10041000100CF602080C2807000C34001802220009
:100420002807180C340077000A0C36001802220046
:100430003503F504200C28062E0C34001802220087
:10044000220C1B0AF505B7022A0C28062E0C3400D4
:10045000180222002C0C1B0A000C1B0AF6000000DC
:10046000360C2807180C340018022200380C310A08
:10047000F6021704400C2807000C34001802220072
:10048000420C3B0A4A0C1707100C2807000C3400DA
:1004900018022200000029053C0A4907550C4806AD
:1004A0003800050C3A001C0222005D0CFA02550CC3
:1004B00048074D0C38001C0222004807650C380024
:1004C0007B000A0C3A001C0222003903F9046D0C6F
:1004D00048067B0C38001C0222006F0C680AF905E4
:1004E000BB02770C48067B0C38001C022200790CFA
:1004F000680A4D0C680AFA000000830C4807650C76
:1005000038001C022200850C7E0AFA021B048D0CA6
:1005100048074D0C38001C0222008F0C880A970CEB
:100520001B075D0C48074D0C38001C022200000020
:100530004905890A6907A60C68063C00050C3E00BF
:10054000A3046403A803A90310022200B20CFE0254
:10055000A60C68079A0C3C00A3046403A803A90333
:10056000100222006807BE0C3C007F000A0C3E000F
:10057000A3046403A803A903100222003D03FD04A1
:10058000CA0C6806DC0C3C00A3046403A803A9039E
:1005900010022200CC0CC10AFD05BF02D80C68066F
:1005A000DC0C3C00A3046403A803A903100222008E
:1005B000DA0CC10A9A0CC10AFE000000E80C6807B8
:1005C000BE0C3C00A3046403A803A903100222008C
:1005D000EA0CDF0AFE021F04F60C68079A0C3C00C6
:1005E000A3046403A803A90310022200FB0CED0A74
:1005F00000006905EE0AF80C1F07B20C68079A0C98
:100600003C00A3046403A803A90310022200C70C42
:1006100002006700EF0C07000F0C3000A40530004B
:10062000000C3400A40434004D0C3800A40538003C
:100630009A0C3C00A4043C00C4050E0C3000690078
:1006400068006A006F00A405010C2C003800390016
:100650003A003B003C003D003E003F000A0C2D00EC
:10066000FA0C2E000000C70C2800A7073E0BE8027A
:10067000350BEE02320BED02300B2F05A304780A86
:0207FE00380CB5
:021FFE00D20F00
:00000001FF
